:020000040000FA
:060000000219FD02031CC1
:03000B0002008D63
:03001300020537AC
:03001B0002009050
:03002B000202D1FD
:03005B0002054655
:030073000203097C
:100080000406080C10182030406080A0C0054032E3
:10009000C2AFC2A853E6EFC28E856B8BC0D0D2D35D
:1000A000C0E0C0F0C2CAA8CCA9CDD2CAD2AF758A6E
:1000B00000C3E8956CF8E9956DF9C3E913F9E81305
:1000C000F8E5666007C3E913F9E813F8E97025E875
:1000D000956E4020956E501CE582B410177C007B15
:1000E000007A007908900000A86AE5667004C3E809
:1000F00013F801FD900000D2A8D2AA61E7E0FDC389
:100100009CC39840EF98EB33FB0582E0FCC39DC392
:100110009840E198EB33FB0582E0FDC39CC3984017
:10012000D398EB33FB0582E0FCC39DC39840C59890
:10013000EB33FB0582E0FDC39CC39840B798EB33DB
:10014000FB0582E0FCC39DC39840A998EB33FB05F7
:1001500082E0FDC39CC398409B98EB33FB0582E093
:10016000FCC39DC398408D98EB33FB0582217890AA
:100170000000D2A8D2AA61E7E0FDC39CC39840EF7B
:1001800098EA33FA0582E0FCC39DC39840E198EAFF
:1001900033FA0582E0FDC39CC39840D398EA33FA52
:1001A0000582E0FCC39DC39840C598EA33FA0582F6
:1001B000E0FDC39CC39840B798EA33FA0582E0FC9F
:1001C000C39DC39840A998EA33FA0582E0FDC39C19
:1001D000C398409B98EA33FA0582E0FCC39DC3981C
:1001E000408D98EA33FA0582EBC46B6A54F0F9EA61
:1001F000C454F0C3996009900000D2A8D2AA61E764
:10020000EBF4C454F0F9EAF4C4540F49FAEBF4C423
:10021000540FFBC3EAF99460FAEB9400FB5020C33F
:10022000E97B007A0079006016C3135006F9C39584
:1002300052600AE9F5527553007900800205533087
:100240003A27C3EA94D0F8EB9407F9400BE8FAE9AF
:10025000FB203509D235415D303502C235203902E7
:10026000B235C3EA33FAEB33FBEB2B3B3BF9C3EB81
:1002700013FBEA13FAEA29FAEB3400FB30E3047AC1
:10028000FF7BFFE5255403601B202A18E55D33F949
:10029000EB7007C3E99A4002E9FAE53CC4332AFA55
:1002A000EB3400FBC3EA33C4540FF8EB33C454F00F
:1002B00048F87005EA60027801900000D2A8D2AA3E
:1002C000E5226002152281D4900000D2A8D2AA6152
:1002D000E7C0D0C0E0C2CF0541E5666009E56560D2
:1002E000057565006104756501E52360021523C38A
:1002F000E55460057555006104E5552401F5555038
:10030000037555FFD0E0D0D032C2AF53E67F75926F
:10031000FA7593FFC22053917FD2AF32C0E0E58AD5
:10032000303408856B8BF0A3D0E032D0E0C2AF53FD
:10033000E6EFC0D0C0E0C0F0D2D3D2AF5388EFA870
:100340008AA98CAA40308D010A758A00758C0075C7
:100350004000438810E566700AC3E833F8E933F9D2
:10036000EA33FA30331FE8C4540FFAE9C454F04AB0
:10037000FAC3132AFAC3E833F8E933F9E82AFAE9A9
:100380003406FB61D830320FC3E833E933FAE82A88
:10039000FAE93400FB61D8303115E875F056A4AAAB
:1003A000F0E975F056A42AFAC5F03400FB61D8C311
:1003B000EA13FAE913F9E813F8E875F056A4AAF07D
:1003C000E975F056A42AFAC5F03400C313FBEA130A
:1003D000FAC3EB13FBEA13FAC3EB94125009C3EA16
:1003E0009434EB940750160522E52270021522C3BF
:1003F000E52294325002A12A755400A12DE5226015
:100400000215223036067C007D088117AC31AD32F2
:10041000303A04AC33AD34C3EA9CFAEB9DFB92084E
:10042000AE60AF61303A425007203509D235813590
:10043000303502C235303504AE62AF63203902B2C6
:1004400035C3EA33FAEB33FBA208500AEAF424017D
:10045000FAEBF43400FBC3EA9450FAEB9400FB503F
:100460001478007A007B008175A208500878007A21
:10047000007B0081D4E5255403601B202A18E55D2C
:1004800033F9EB7007C3E99A4002E9FAE53CC4335B
:100490002AFAEB3400FBEA8EF0A4F9AAF0EB8EF016
:1004A000A42AFAC5F03400FBC3EB13FDEA13F8C32A
:1004B000ED13FDE813F80FEF146004C3E833F8C33D
:1004C000E933EA33FAEB33FBDFEDEB30E30678FF99
:1004D0007AFF7B078854D230E86003755500C3E586
:1004E0005BFC955C4002AC5CC3EC95545008EC7529
:1004F000F008A4FAABF0EAF4F8EBF45407F98856E4
:10050000895775230AE55A30E210D0F0D0E0D0D0F8
:1005100053F7DF43F74043E61032D0F0D0E0D0D0BD
:1005200053D8FE43DA0143E6103275230AD0F0D0E7
:10053000E0D0D043E61032C2AAD28EC2CA85CC6CBB
:1005400085CD6DD2CA32C2AFC0D0C0E0D2D38556FD
:10055000FB8557FC85575A53F7BF53DAFED2A830B4
:100560003402D2AA53E6EF53F7DF53D8FED0E0D0DF
:10057000D0D2AF327901801479038010790A800CCF
:10058000791E80087964800479C880007817E4D5E2
:10059000E0FDD8FAD9F62278FF20282879A1E76073
:1005A00023E548601F74FF8548F084853FF03029BB
:1005B0000375F005A4F8C5F0600278FFC3E8955D07
:1005C0005002A85D885C22C3E54794A0E5489400EA
:1005D000E55C500314A1D8046002F55C2275E89034
:1005E00022055EC3E55E9408405330EDF4A8BDA932
:1005F000BE755E00E9FA79A0E76041EA7006E55F42
:100600006018800CC3E8955F600EE55F5005600AD6
:100610001480070460FA8002E55FF55FC3956940C6
:100620001B755BC0C394044013755B80C394044086
:100630000B755B40C394044003755B0022E55B24AB
:1006400010500274FFF55B22743279A687F0A4C5BE
:10065000F0A2F733F55D227547007548F022C2AF6E
:10066000C2CAA8CCA9CDAA4130CF010AD2CAD2AF02
:10067000C3EA13FAE913F9E813F8AB42AC43884232
:100680008943C3E89BF8E99C20280A547FF9302C61
:1006900002E17CC1D5AD448A44F9EA9D547FFA60F9
:1006A0000678FF79FFC1BAAE45AF468B458C46A8A8
:1006B00042A943C3E89EF8E99FF9C3E54813FBE567
:1006C0004713FAE82AF547E93BF54850067547FF16
:1006D0007548FFE122AA47AB48AC47AD487E047F8E
:1006E00002C3EB9404400D1E1FC3EB940840052089
:1006F00029021E1FC3ED13FDEC13FCDEF7C3EA9CB9
:10070000FAEB9DFBEF6009C3E913F9E813F8DFF793
:10071000EA28FAEB39FB8A478B4850067BFF8B4768
:100720008B48C3EB94025002D22C3028047F03E1A3
:100730004D7892E6FFC3E53D948240110FC3E53D3D
:1007400094A040010FC3EF940640027F057E02E5AE
:1007500048C4540FF9E548C454F0F8E547C4540FB1
:1007600028F8C3E89EFAE99400FB4009C3EA940123
:10077000EB940050047A01E4FB0207C8AA47AB4897
:10078000EBC4FEEAC4540F4EFCC3EA9CFAEB94009F
:10079000FBC3E813C313F8EA28FAEB3400FB8A47DB
:1007A0008B48C3EB94024002C22C7802EBC4FE7B60
:1007B00000EAC4540F4EFAC3EA98FA4005C3940104
:1007C00050027A017892E6FF302002E1C8854E920D
:1007D000854F93D22043E680C3E49AF8E49BF9C3A3
:1007E000E833F8E933F9302C0302085DE8FAE9FB55
:1007F000D3E913FDE813FC884E894FC3EF940360DF
:1008000038EF20E00CE82CF8E93DF9ECFAEDFB803C
:1008100013E828F8E939F9C3E82401F8E93400F9C4
:100820007AFF7BFFC3EF9403400F8A508B51884AB5
:10083000894B8C4C8D4D020892885089518A4A8B85
:100840004B8C4C8D4D3028127550F07551FF754C06
:10085000F0754DFF754EF0754FFF020892E8FAD320
:10086000E813FC884EC3EF94036021EF20E007E813
:100870002CF8ECFA017DE8282401F87AFFC3EF9404
:100880000340098A50884A8C4C02089288508A4A50
:100890008C4C3020020192753A02D22043E680E56A
:1008A000255403602DA847A948C3E913F9E813F8B4
:1008B000302804E92440F9C2AF53E67F759100C3A4
:1008C000E498F594E499F595759104D22043E68077
:1008D000D2AF22D221754900752000302B0375203C
:1008E0004001F1D221754900752040302B0375205D
:1008F0000078017901202C20E52554036002C221F3
:100900007914E548C313700104F8C39414400278C5
:1009100014302804781B791BC3E833F8C3E933F992
:10092000202010E549600C302803D53A04D222215A
:10093000A4119A0549E59B5440B52002218E302828
:100940000908C3E899400118212020210A08C3E8BA
:1009500099400201F12120C22153E67F75910030B8
:100960002C117594007595F0759104D22043E680A2
:100970000208F1E5487EFFC3334009C3334005C395
:10098000334001FEC3E49E759400F5952168C3E5EC
:10099000399401500201F130210201F1D80221A263
:1009A0002120C222C2AF53E67F7591008550948505
:1009B0005195759104854A92854B93D22043E680E8
:1009C000D2AFE52554036007202902053980103095
:1009D000220D202B0A202107158115810213D52213
:1009E00078003021027801E53D75F007A4F9E5F0C3
:1009F00028F5F0E9A2F013A2F113A2F213F53DC31A
:100A000094785003753D78C3E53D953E4009C29406
:100A1000C292C29075D53F3020024117854C928515
:100A20004D93D22043E68022203814C2AFC292C236
:100A300095D294D29075D53DD2AF759F206128C2D2
:100A4000AFC292C291D290D29475D51FD2AF759F8A
:100A5000206128203814C2AFC290D29275D537C217
:100A600095D294D2AF759F306128C2AFC294D29212
:100A700075D537C291D290D2AF759F1061282038BA
:100A800014C2AFC294C291D290D29275D537D2AF70
:100A9000759F106128C2AFC290C295D294D2927550
:100AA000D537D2AF759F306128203814C2AFC292BB
:100AB000D29475D51FC291D290D2AF759F20806815
:100AC000C2AFC292D29075D53DC295D294D2AF75C5
:100AD0009F208054203814C2AFC290C293D292D2C9
:100AE0009475D51FD2AF759F30803DC2AFC294C2FE
:100AF00093D292D29075D53DD2AF759F10802920A8
:100B00003814C2AFC294D29075D53DC293D292D25E
:100B1000AF759F108012C2AFC290D29475D51FC21C
:100B200093D292D2AF759F30227A147B7880127A5A
:100B3000107B8C800C7A0D7BB480067A0B7BC8808E
:100B400000E564D5E001227902E4C292D5E0FDD24D
:100B500093D292D5E0FDC292D5E0FDC293D292D558
:100B6000E0FDE920E004D295D29430E004D291D2A5
:100B700090E564D5E0FDE920E002C29430E002C2D5
:100B8000907496D5E0FDD9C1EAF8D5E0FDD8FBDB3D
:100B9000B0C29222C294C292C290C294C292C29037
:100BA00075D53F22788076FF0876FF0876FF0876B5
:100BB000FF0876FF0876FF0876090876FF087601B9
:100BC000788C76010876FF0876FF0876FF0876FFB6
:100BD0000876FF0876030876FF0876FF0876FF0898
:100BE00076250876D00876280876500876040876A8
:100BF000FF0876020876FF08767A0876FF087607FF
:100C00000876010876FF0876FF087600087600224D
:100C1000FA75F00CA4ABF0EAC333F8740133F9E8C9
:100C2000C333F8E933F9E8C32BF8E93400F9E8C332
:100C300033F8E933F9227888E6C39403D23A5002B4
:100C4000C23AC238E630E102D238A2389239788608
:100C5000E6149000809378A6F67886E6F53FC39474
:100C6000025003753F02789CE6753EFFB40203759F
:100C70003EA0B40303753E8278A0E6F860067428AF
:100C80002409D8FCF5697896E69110883189327884
:100C90009EE69110883389347897E69110883589DB
:100CA000367194223036117A007B007CFF7D007E05
:100CB00000B10A8B618A6022303A227896E6FA7B8C
:100CC00000789EE6FC7D00C3EA33FAEB33FBC3EC0D
:100CD00033FCED33FD7E0AB10A8B638A627896306D
:100CE0003A02789EE6FA7B007897E6FC7D007E006B
:100CF000303A10C3EA33FAEB33FBC3EC33FCED3389
:100D0000FD7E0AB10A8B618A6022C3EC9EFCED94E1
:100D100000FDC3EC9AFCED9BFDC3EC9423ED940025
:100D200050047C237D00C3EC94FFED940140047CCF
:100D3000FF7D017BFF0B7A000AEA7009C3EC33FCEC
:100D4000ED33FDA135EC8AF0A4AEF0ED8AF0A42ECF
:100D5000947C40E4EAF460DD22D23691A41205804E
:100D60001205807A007B007C10120578E5542AFA7F
:100D700074003BFBDCF37C04C3EB13FBEA13FADCEB
:100D8000F7FFEB60027FFFC23691A42278A5E6F957
:100D900054037000E9540C7000E954307000E954B9
:100DA000C07000227567007568007597DE7597AD95
:100DB0007581C043FF8075EF0675A9007194758039
:100DC000FF75F1F075A4007580FF75D4FF75900074
:100DD00075F23F75A53F75900075D53F75A60175F5
:100DE000E34075E2027194E4F8F6D8FD71A41214A0
:100DF0001F78988664753001C2AF12058871291278
:100E00000580712F1205807135120580B18CC2AF3B
:100E100075670075680078FA79FA308507D9FBD8CC
:100E2000F7021C00913691A478988664719475A994
:100E30001375A71075C10075A70075660075E405E8
:100E4000758811758E0475890975C80475910475C6
:100E5000D84075D90875F783759E0075960075DAC8
:100E60004A75DB0075A82375E69075B801759B80FF
:100E7000759D0075D10C75BCB975BB1075E8807592
:100E8000B201120574D2AF753C00C230120588C29F
:100E900031C232C233C23475520075220012058449
:100EA000C3E522940A5002E171D231752200120585
:100EB00084C3E522940A5002E171C231D232752214
:100EC00000120584C3E522940A5002E17175E4D54D
:100ED000758851758E017589AA758C00758D00C253
:100EE000A9D2ABD2AA756B80756A14756E50C232E6
:100EF000D23475220A120584756A10C3E522940A59
:100F00007552007553004069758E0C756B00756ADB
:100F100028756E2875220A120584756A20C3E52299
:100F2000940A7552007553004047758E0C756B809E
:100F3000756A14756E1475220A120584756A10C3D9
:100F4000E522940A755200755300402575E4057535
:100F50008811758E04758909D2A9C2ABC2AAC234A0
:100F6000D233752200120584C3E522940A4002C1DF
:100F70000E120578203003020E0EC2AF71297129BE
:100F80007129D2AF120588203403303A030210329F
:100F9000120578788CE6C394015003021032E530D4
:100FA000C3940150030210327567A57568F17F0282
:100FB000D23691A4120584C2AFC23691A4C3E554BF
:100FC000947FD2AF406C120574C2AF713BD2AFDFD9
:100FD000DFB159C3EF7897F612058812150C7F0A16
:100FE000D23691A4120584C2AFC23691A4C3E5548F
:100FF000947FD2AF50E8120574C2AF712912057CFC
:10100000120B29D2AFDFD9120D59EF24037896F6CF
:10101000F87997E7C394234003985006E82423788F
:1010200097F61205889166B13B120584120CA40252
:101030000E0E756700756800120584C3E5549401AF
:101040004003020F87C2AF120B3B120B3B120B3B4C
:10105000D2AF120588753000E4F537F5380537E56D
:1010600037F4703F0538789AE678191460127832B0
:1010700014600D787D14600878FA146003753800E8
:10108000C3E53898401D120B941205741538753756
:101090000078998664C2AF120B3BD2AF7898866411
:1010A00012058412057CE5237003020E0EC3E5527F
:1010B00094015014C3E554940140A2120584E52321
:1010C0007003020E0E021266C3E55294017017C23D
:1010D000AF120B9478998664120B2978988664D2A3
:1010E000AF1205844158C3E55294027017C2AF1283
:1010F0000B9478998664120B2F78988664D2AF127D
:1011000005844158C3E55294037017C2AF120B9483
:1011100078998664120B3578988664D2AF1205846C
:101120004158C3E55294047013C2AF120B947899DE
:101130008664120B3BD2AF1205844158C3E552942A
:10114000057017C2AF120B9478998664120B3B7826
:10115000988664D2AF1205844158C3E55294077053
:1011600019C3E5539409500201AD7401303A027479
:10117000037888F6C238C2394158C3E552940870E2
:1011800019C3E5539409500201AD7402303A027458
:10119000047888F6D238D2394158C3E552940970A0
:1011A00017C3E5539409500201AD303A0BC3788858
:1011B000E69402F6C23A4158C3E552940A7016C347
:1011C000E5539409500201AD203A0A7888E62402DA
:1011D000F6D23A4158C3E55294147025C3E55394AE
:1011E00009500201ADC2AF901A0B740093D2AF78D0
:1011F00088F613C238C2394002D2384002D2398050
:1012000057C3E55294157038C3E5539409404FC253
:10121000AF901A0B740093D2AFF8B801027402B801
:1012200002027401B803027404B8040274037888DB
:10123000F613C238C2394002D2384002D23980187F
:10124000C3E552940C70117567A57568F1C3E55339
:101250009409400A9166D2AF7552007553007567C4
:101260000075680001ADC2AF120B94E4D2AFE4F593
:101270005EF524F525F53D755E081205741205DD51
:1012800030EDFDA8BDA9BEE97001F8885F1205E147
:10129000755E08C2AF120648855D5B855D5CD2AFA6
:1012A00075A71075C13075A70075A9037566013063
:1012B0003A07C238303502D238D228753900120ABE
:1012C000D4120AFF12065712065E12065712065E65
:1012D0001206571208E31209E0120A2812065E12DB
:1012E00008D3202C03120597302C031205C71209CE
:1012F000E0120A5312065E1208E31209E0120A7E97
:1013000012065E1208D31209E0120AA912065E1232
:1013100008E31209E0120AD412065E1205DD120873
:10132000D31209E0120AFF1205E112065E302827E7
:10133000855D5B79187A0CC3E53999400EC228D2D5
:10134000298A3B855D5B855D5C800CC3E554940117
:1013500040030212D361DD30291F202B1CE53B1412
:101360007006C229D22A41D3F53B203A07C3E5547F
:10137000940140030212D38064753C00203A0F7838
:10138000FA79A4E760027803C3E55598504FE52346
:10139000604B303A17203805203507800F30350272
:1013A000800A202B07D22B855D5B610378F0302B00
:1013B00005855D5B7820C3E5489850030212D33061
:1013C0002B1BC22BC238303502D238D229753B12C2
:1013D000855D5B41D3053CE554600261E0753C00EE
:1013E000C2AF120B9475240075250075A91375A75B
:1013F0001075C10075A700756600D2AF1205841282
:101400000B9478A4E6600CC295D294C293D292C297
:1014100091D290C3E53C94044003020E0E01589013
:101420001A0D7820919FE520B4550AA3919FE520DD
:10143000B4AA0280137567A57568F1120BA49166B2
:10144000756700756800801D901A0378807B0A918B
:101450009FA308DBFA901A0F788C7B1A919FA30840
:10146000DBFA901A2922C2AF91E291BF901A007460
:101470001091A4A3743E91A4A3742191A4901A0383
:1014800078807B0A91A3A308DBFA901A0F788C7BF3
:101490001A91A3A308DBFA91F591D3901A2922E4BB
:1014A00093F622E6438F01538FFDFFC3E583941C1F
:1014B000400122EF8567B78568B7F0538FFE22435E
:1014C0008F02438F018567B78568B7901A0DF05377
:1014D0008FFC22901A0D745591A4901A0E74AA9143
:1014E000A4227A3079D07820901A40919FE520F795
:1014F00009A3DAF7227A3079D0901A40E791A4094B
:10150000A3DAF9227C05120588DCFB22C2AF120B9C
:1015100029120B2F120B35120B3B12057C120B29D3
:10152000120B2F120B35120B3B12057C120B2912DA
:101530000B2F120B35120B3BD2AF22C2AF120B3B5B
:10154000120B35120B2F120B2912057C120B3B12BA
:101550000B35120B2F120B2912057C120B3B120BB1
:0A15600035120B2F120B29D2AF2217
:1019FD00020DA4103E21FFFFFFFFFFFF09FF01FFB6
:101A0D0055AA01FFFFFFFFFF03FFFFFF25D0285061
:0D1A1D0004FF02FF7AFF0701FFFF0000FF3A
:101A400023425F485F3030232020202020202020A8
:101A500023424C48454C492445464D3842323123B7
:101A60002020202020202020202020202020202076
:101C0000C2AFC2D37597DE7597AD7581C075A90057
:101C100043FF80752438752503B1DB7529A5752A26
:101C2000F143F12053A4DFD28575D4FF75E3407DE5
:101C3000FA780379E67C10752200752300901DE880
:101C40007B0675249875250130850281482085081A
:101C5000D8FBD9F9DCF781BA308508D8FBD9F9DC93
:101C6000F781BAB19BE493A3C39A6004DDC381BA40
:101C7000DBDBB18D600281317B08E493FAA3B16EA6
:101C8000DBF87A30B16E752200752300B18DEAFC65
:101C9000EBFDC3ED94FE400EB18D8A278B28ED300D
:101CA000E0048A828B83B18D7AC270D8C3ED94FE32
:101CB000601950CEBD0029EC600F7520007521FF22
:101CC000752900752A000200008100A827A92808AC
:101CD00009D804D90281DDB191EAF281D10D81A642
:101CE000C3ED94035051EDA2E092007AC5C3E582A2
:101CF0009400E583941C508C200010438F02438F86
:101D0000018529B7852AB7F0300027A827A9280818
:101D100009438F01538FFDD804D902A132C3E58353
:101D2000941C4003A3A117E28529B7852AB7F0A325
:101D3000A117538FFC81827AC1BD030CE493A3FAEF
:101D4000B152DCF8B14A81828184AA22AB23B16E00
:101D5000EBFAEA6222752608C3E52313F523E52290
:101D600013F52250066323A0632201D526EAB1DBD6
:101D7000B1DB75260AEAF4200102D285300102C2E5
:101D800085B1DBC3134002C201D526EB22B191EA33
:101D9000FB208502A191308502A196752608AE240C
:101DA000AF25C3EF13FFEE13FEB1DFB1DBC3EA13C0
:101DB0003085024480FA30E703632201C3E5231330
:101DC000F523E52213F52250066323A0632201D5F3
:101DD00026D9E52265236523F52222AE24AF250E00
:101DE0000FDEFEDFFCD20122424C48656C693437BD
:061DF0003164E8B20601B7
:00000001FF
